:030000000201CD2D
:0C01CD00787FE4F6D8FD75811A0200036B
:10000300751001E4F517F50CF50D7515FFF516756B
:100013008911758810F5B0E59030E7100517D3E521
:10002300176480948440087517058003E4F517E48A
:10003300F50EF50F858A18AF8CEF250FF50FE43514
:100043000EF50EE50F750F00F50EE518250FF50FEC
:10005300E4350EF50EC3E50F950DE50E950C401036
:10006300AF0DE50DF50DEF6007E510700343B0012B
:10007300D3E50F94F4E50E9401400DE50F94D0E51C
:100083000E9407500353B0FCD3E50F9400E50E9490
:10009300FF4003751001E58C30E70543B080800312
:1000A30053B07FE5176404600302001AF58AF58CE8
:1000B30043B003E5106003020196F50BF50AF50959
:1000C300F508FCFDE50B250FF50BE50A350EF50AE2
:1000D300ED3509F509EC3508F508AE15AF16AB0794
:1000E300AA06C3E50B9BF50BE50A9AF50AE5099405
:1000F30000F509E5089400F508850E15850F16E44B
:10010300850F14850E13F512F511FFFEAB0BAA0A2A
:10011300A909A808D31201A64018E514250BF51464
:10012300E513350AF513E5123509F512E51135081E
:10013300F511AF907519008F1A631AFF6319FF53F6
:100143001A3C751900E51AAE197805C333CE33CEC0
:10015300D8F9F51A8E19FBAA06C3E5149BF514E525
:10016300139AF513E5129400F512E5119400F511B5
:10017300E4FF7E80FDFCAB14AA13A912A811D312CD
:1001830001BC4007E4F50CF50D801285130C8514B2
:100193000D800AE4F50CF50D7515FFF516E4F51061
:0301A30002001A3D
:1001A600EB9FF5F0EA9E42F0E99D42F0EC6480C8D0
:0601B60064809845F02270
:1001BC00EB9FF5F0EA9E42F0E99D42F0E89C45F099
:0101CC002210
:00000001FF
